:1074000080E189BD82E189BD09B400FEFDCF089508
:10741000AA2069F08091E9008F931092E900ACD422
:1074200083FF01C02BD58F9187708093E900089569
:107430008EEF0090E10008220092E1000895F20131
:10744000F999FECFF2BDE1BD0895F9DFF89A80B554
:1074500008C0F5DF1FBA80BD0FB6F894FA9AF99A02
:107460000FBE31962F010895E0E0F0E085919491F0
:10747000019608958BEA34D0109289008AEF8093A8
:10748000880082E080936F0083E080938100E1EACE
:10749000F7E785913AD0ED3AE1F781E08093D700A4
:1074A0008AE482BF1092D8001092E2001092DA00B3
:1074B0001092E10080E808D019BCAA241092E000E4
:1074C00071D489E062D481E98093D8000895A3E65D
:1074D000B1E090E81AD08D939A95E1F7089586E08F
:1074E00008D010C083E005D08F2F0FD08E2F0DD085
:1074F00080E05E9A729809C005D085E0FADF05D079
:1075000080FDFDCF729A5E9808958EBD8DB587FF80
:10751000FDCF8EB508958FE08221E9F7F3DFE3E632
:10752000F6E090EB5C98892FF0DF80E1EEDF5C9A6B
:107530008191EBDF83E68E278F77D1F79395983B88
:1075400089F70895E3E6F1E097FC36C094FC4DC05E
:1075500092FE089596849920D1F3F894C089D78536
:1075600020E030E080E090E4AFEFBFEF11968919A2
:107570009040E0F72D01BD4F8D0127FD13C0E0E0E5
:10758000F8E011928EE7819392E4E11791939AE5E6
:1075900008F092E4E334C9F781931082BFDFFE0163
:1075A0002196A0DF94DFF9010BD520583F4F040D41
:1075B000151D9A9411F70FC28301282D60906C015C
:1075C00070906B0143D019F48823C1F708953801F6
:1075D00088243CD0C9F580916A01821709F483019F
:1075E00060906E0170906D01F4CF80E1982E6090F4
:1075F0006E0170906D012AD059F48823B1F7089577
:107600009FEF95FC03C096FE089591E097FB890ECD
:10761000662477248301222719D0B1F48823A1F3AB
:1076200080916A0136F0881650F4821730F02130CC
:1076300003C0881520F4281710F48301282F6090C8
:107640006E0170906D01E8CF3801822EF3014ADFA0
:107650003EDFC3E6D1E0EAE9F7E709908591081635
:1076600021F4E13AD1F7088080104CCFC9E031DF36
:10767000CA95E9F7D0E195FC1FC094FC38C096FC90
:1076800001C051C0C3E6D2E0E3E6F6E098E088E747
:107690008E0F00840192E817E1F7884F099001925C
:1076A000E817E1F7C858DF4F9A9589F734DFC85FCC
:1076B000D340C33E49F749C0C3E6D6E0EBE5FAE064
:1076C00098E08E2F885702900086E817E1F73896E9
:1076D0000A900292E817E1F73897C857D0409A9578
:1076E00081F719DFC850DC4FC33E41F72EC0A3EE2F
:1076F000B6E0E3E6F6E09AE0C6E00D9080818025F2
:10770000807F802582958193A336B90709F4B2E082
:10771000E336F90709F4F2E0E336FC0771F7FBDE24
:10772000DA9529F712C0A3EEB9E0E3E6FAE092E0B9
:107730000E90829180258F70802582958083E3361C
:10774000F907B1F7E8DEDA9571F78827089580E840
:1077500080BF8DEA8093640089E98093650085E0AD
:1077600083BF8895E8EBF0E081818C7F81838CE09A
:10777000808374E0720D84EA02C0838384E884838A
:10778000848187FD08957211FBCF089502D084E9AA
:10779000848388E08A95F1F7089541524455424F19
:0E77A00059D5F08D14A1C881CFD9F1AF0000EA
:1077AE001201100102000008412336000100000002
:1077BE00000109023E0002010080320904000001AE
:1077CE00020201000524001001042402040524060F
:1077DE000001070582030800FF09040100020A00E8
:1077EE0000000705040210000107058302100001C6
:1078000011241FBE04B714BE88E18093600010925B
:1078100060008EEF9AE09EBF8DBF222433242101A9
:107820003101410180E887C00F928F939F931F928F
:107830000FB60F9211244F936F938091DA0080FF5F
:1078400034C020C00F920FB68F939F93EF93FF9396
:1078500088278093850080938400E0E5F1E09081A3
:107860008917980B908309F45D9A91818917980B79
:10787000918309F4289A239411F48315381EFF91FB
:10788000EF9154C08091D80080FF0FC08091DA0042
:107890008E7F8093DA008091D90080FF04C0B0DD34
:1078A00081E0A82E02C019BCAA248091E10080FFCB
:1078B0000BC065D280FF08C065D28091D80080627D
:1078C00003DE19BC85E0A82E8091E10084FF1AC078
:1078D00056D284FF17C094DD8091D8008F7DF4DDEF
:1078E0008FEEA7DD4CD28F7E81604FD28091530105
:1078F000882331F48091E30087FD02C081E001C05C
:1079000084E0A82E8091E10083FF0CC038D283FF71
:1079100009C087EF8EDD82E0A82E1092530188DD2A
:1079200031D240D26F914F910F901F909F918F91C4
:107930000FBE0F9018958093610010926100B1E026
:10794000B5BF82E085BF81EF85B987EE84B984E059
:107950008DB984E48EB910BA83EF81BB80E68BB910
:1079600080EF8AB980E58CBDBDBDA0E0EEEAF7E707
:1079700005900D92A035E1F78C911D92BB30E1F797
:10798000893B11F4ADDDE3CE5F9A04C07C9B02C05D
:107990006BDD09F56FDD789459DEB4D039DD8FB138
:1079A0008095807F66991C9B8460982E29DE89EBE8
:1079B00088258093FF0A8110C5DD92FC0AC08FE004
:1079C0008221882921F48091720187FF19D0332008
:1079D00022F74ADD11F3F89489EB82DD81E0809390
:1079E000E00010926F0010928100109285001092BA
:1079F000840081E085BF15BE5D9A289A0C94000032
:107A0000E5E0F0E06FDDA3E6B2E0C8E062DDCA9534
:107A1000E9F7A8DE80EDB1DE80E0AFDEB7DEABDEF9
:107A200081EDABDEC4E7D1E0DE0184ECA8DE83812A
:107A30008D93AA37D1F7A2DE83818D93A7DE1482BE
:107A4000AFE2B6E08D8117D08C8115D08E8113D036
:107A50009A8190748A8119F08F7184FF80560BD0BF
:107A6000898109D0888107D0992321F08A81869560
:107A7000807102D053CD00D09E01DD91CD91CD59C2
:107A8000D94FFD91ED91ED59FE4F41915191549F88
:107A90008295682F6F70609DE00DF11DBE01152E5F
:107AA0008E0103561640143050F401900882C058DD
:107AB000DF4F1A94A9F7EB0121964A9579F7E9016E
:107AC000089558D107C009D102C0AA2039F054D175
:107AD00082FFFBCF85FFF7CF8091F1000895082E3C
:107AE00083E049D185FD07C03ED102C0AA2049F0FC
:107AF00043D180FFFBCF0092F1005D9884E6809334
:107B00005001089537D182FFEAC0289884E6809317
:107B10005101D7DF182F853431F422248EE7382E17
:107B20008EDC8DE0C5C0843511F4CBDFFACF8C3408
:107B3000C1F38035B1F3843711F480E0B9C08134EA
:107B400029F4BFDF582EBDDF482EEBCF833539F443
:107B5000EAE9F7E78591C3DFE13AE1F7AAC08635A4
:107B600021F482E3BCDF81E3A3C08A3649F48FE9C4
:107B7000C0DCC3E0CADCB3DFCA95E1F7C3DC99C05F
:107B8000833731F487E8ABDF85E9A9DF8EE190C068
:107B9000823631F489E5A3DF80E0A1DF80E888C088
:107BA000823419F0873609F06FC033248ADFD82F6A
:107BB00088DFC82F86DF082F8354843008F077C011
:107BC000063411F4440C551CF20110926F00173664
:107BD000B9F4033489F483E086DC97DC8EB51EBCEF
:107BE0007EDF0DB42197D1F78DDC08C0063411F487
:107BF000859101C02ADC73DF2197C2F72F013CC0B9
:107C00000334A9F4E11104C06ADC88ED6CDC74DC97
:107C100066DC82E068DC55DF0DB48EBDCA95D9F70D
:107C2000319674DC69DCDA9569F72F0123C00634DC
:107C3000C1F49F01F437A8F4D6D113C042DF063453
:107C400061F4C0FB46F0F43728F4182E81E087BFBA
:107C5000E89511243296082E04C0043409F401C0BA
:107C6000F8DB21975AF7063429F42F01F901F4378C
:107C700008F4B7D18DE033DF063411F456944794FD
:107C800082E080936F0015C08237E1E049F08634CE
:107C9000E0E031F08E34E3E019F0813531F4E2E0D8
:107CA000F0E089E087BF849103C08B3111F08FE34E
:107CB00016DF83E0BADB57D095FF03C009C0AA20C6
:107CC00071F05AD080FFFBCF4ED002C0AA2039F00D
:107CD00053D080FFFBCF84E0A8DB8BE745C008953D
:107CE000E4E5F1E067E090915B0180915C01913205
:107CF00031F0913AF1F58132E1F560D183C0823201
:107D000081F48191805B8191844099F580915D013E
:107D100080FD2FC0F89481E08093E0001092FF0A6C
:107D20006FCD803231F54AD1AA20E9F08530D9F003
:107D300023D083FD18C082FFF7CF04C0CDDE81932E
:107D4000615031F09091F3008091F200892BB1F7EE
:107D5000C4DF611549F704C0AA2029F0853019F065
:107D60000BD080FFF9CF8EE79091E80089238093B4
:107D7000E800089584E059DB8091E800089580913F
:107D8000E2000895FCDF8E7F80618093E200089519
:107D900082E061EC09D083E061E802D084E060E831
:107DA00042E103C080E060E042E03FDB81E007D0D9
:107DB0001092ED006093EC004093ED0008959091D7
:107DC000EB00892B8093EB00089560E0923029F05E
:107DD000913029F4E0E062E102C0E2E16EE3F1E01B
:107DE000089580915B0188234CF402C0AA20C1F35E
:107DF000C3DF82FFFBCF71CFAA2091F3BDDF80FFED
:107E0000FBCFB1CF409161015091620146175105FE
:107E100020F0462F611509F4A6DF50E022C0AA2009
:107E200061F1853051F1A8DF83FD57CFA5DF82FDD9
:107E300021C080FF16C03091F3002091F20006C0EF
:107E400081918093F10041502F5F3F4F411519F010
:107E500028303105A8F350E02830310509F451E00D
:107E600082DF4115E1F65523D1F604C0AA2029F09E
:107E7000853019F081DF82FFF9CF2FCFEBE5F1E0FC
:107E80002BDE8193E336E1F72BDF76DF83FF91C0B2
:107E900080915B0190915C01913009F170F0933019
:107EA000F1F0953009F444C0963009F456C098308A
:107EB00009F460C0993059F767C0823841F7809162
:107EC0005F01B2DA2091EB001092E90077D02295A1
:107ED000269521702093F1001092F10052C0882362
:107EE00011F08230A1F68F71823089F680915D01A8
:107EF0008823D1F420915F01277049F22093E90093
:107F00008091EB0080FF10C0933011F480E20BC031
:107F100080E155DF81E0880F2A95E9F78093EA0038
:107F20001092EA0088E04BDF1092E90047D02AC0A7
:107F3000882391F410915D0110680FB7F8943ED03A
:107F400050DF1ADF80FFFDCF1093E300103883E08D
:107F500009F482E0A82E0FBF2CC08058823048F56B
:107F600080915D0190915E0130DF603011F126D08B
:107F700049DF1FC08038E9F421D0809153018093FC
:107F8000F100F1DE2EDF15C0882399F490915D0198
:107F9000923078F49093530111D023DF80915301F4
:107FA000882321F48091E30091E087FD94E0A92EDD
:107FB000EFDEE2DE83FF089580E201DF87EFD4CEBB
:107FC000A3E6B1E0F437B8F40ED090E40D901D9024
:107FD00081E087BFE89532969A95C1F71124E05861
:107FE000F04085E001C083E001D081E187BFE895E2
:087FF00007B600FCFDCF089567
:067FFA003231E3CFFBDC95
:040000030000740085
:00000001FF
